:10000000689D001001020000090200000B020000C0
:100010000D0200000F020000110200005656FFEF13
:1000200000000000000000000000000013020000BB
:100030001502000000000000170200007902000015
:100040001B020000250200001B0200001B02000032
:100050001B0200001B0200001B0200001B0200002C
:100060001B0200001B0200001B0200001B0200001C
:100070001B020000000000001B0200001B02000029
:100080001B0200001B0200001B0200001B020000FC
:100090001B0200001B0200001B0200001B020000EC
:1000A000912500001B0200001B0200001B02000043
:1000B0001B0200001B0200001B0200001B020000CC
:1000C0001B0200001B0200001B0200001B020000BC
:1000D0001B0200001B0200001B0200001B020000AC
:1000E0001B020000DFF80CD003F038F9004800478D
:1000F0008B090000689D0010D0F800D0D0F804F003
:1001000070B50023084D0AE0CE5C048886EA142608
:1001100035F8166086EA042404805B1C9BB2521EEC
:1001200092B2F1D270BD000070370000FFB50446F6
:1001300029A090E8E000C0688DE8E0000390022963
:1001400002DA002004B0F0BD6018002100F8011DA3
:100150006946B3FBF2F502FB15354D5D00F8015D14
:10016000B3FBF2F3A042F4D8ECE710B502F0BBFB0E
:1001700002F081FD1C4948604FF480520A60A0F5EE
:10018000F420886010BD70B5034608460024164967
:10019000851849688D4200D9881A194603F08FF8EE
:1001A000204670BDF8B50346104600240A460E4DA1
:1001B000161869688E4200D90A1A0090286802F061
:1001C00027FC2046F8BD10B5034608460024194612
:1001D00002F007FF204610BD303132333435363758
:1001E0003839414243444546B400001002E008C893
:1001F000121F08C1002AFAD17047704744332211F8
:100200000648804706480047FEE7FEE7FEE7FEE7B0
:10021000FEE7FEE7FEE7FEE7FEE7FEE74118000027
:10022000E500000010B54FF040210120086001F00A
:100230004BFD10BD10B54FF0E0241A4860611F213E
:10024000601700F01EF80020A0610720206110BD9B
:1002500010B51548022141600021016741611D224E
:10026000C260C16301214160FFF7E4FF0221C81EA3
:1002700000F007F8002010BD0C480168491C01601F
:100280007047C906090E002806DA00F00F0000F1D9
:10029000E02080F8141D704700F1E02080F8001481
:1002A00070470000BFD4010000000940E8000010C2
:1002B00010B50B4604461146184603F03BF8C4E956
:1002C000000110BD40EA01039B0703D009E008C903
:1002D000121F08C0042AFAD203E011F8013B00F80B
:1002E000013B521EF9D27047002001E001C1121FEC
:1002F000002AFBD17047000000000000FFFFFFFF55
:1003000070B52D4C607800282DD000252B4E01288B
:1003100010D002280DD1B0686168401A284988427F
:100320001BD32848406B400017D5012002F00AF883
:10033000657070BDB0686168401A23498842F8D37F
:10034000002001F0FFFFB06860600220607025703F
:10035000BDE870400C2001F0A1B82570BDE87040E8
:100360000C2001F09BB820780028E2D101202070F9
:10037000BDE870400D2001F091B8002802D10E496F
:1003800001204870704710B501F0C4FC0A490020F4
:10039000487010BD084801214170084989684160D2
:1003A000704770477047022803D0032803D100F03C
:1003B00098BE00F0B5BE704718010010000009405B
:1003C000A08601000080092040420F0030B50B4696
:1003D000014600202022012409E021FA02F59D4275
:1003E00005D303FA02F5491B04FA02F52844151E49
:1003F000A2F10102F1DC30BD0000000000000000AD
:1004000000000000AA08000010B5FA4C60698004E2
:100410000CD4F948816843F6982283685B1A9342AA
:10042000FBD36069800401D4012010BD052001F0D8
:1004300035F8002010BD2DE9F0410024EE4EB568DE
:10044000042001F02BF8ED4F02E0FFF7DDFF30B1A3
:10045000B068401BB842F8D3012C02D00CE0012454
:10046000FAE7022404E0FFF7CFFF08B1032403E01A
:10047000B068401BB842F6D3032C02D00020BDE880
:10048000F0810120FBE72DE9F041092001F006F899
:10049000DB48002606704FF47A77C821384601F011
:1004A000F1FBD54CA16842F21075A068421AAA422D
:1004B000FBD3C821384601F0E5FBA168A268501AB9
:1004C000A842FBD3C821384601F0DCFBCC48401CD5
:1004D000867002214171C670D1E70021425C12B9D9
:1004E000491C1829FAD3182901D00020704701208F
:1004F00070472DE9FC4107460E46904600200190CA
:1005000000240EE0351B402D00D9402539192A461C
:10051000BC48FFF758FEAAB2BA4901A8FFF7F0FDA0
:100520002C44B442EED3391942466846FFF74BFEDD
:10053000BDF80400BDF80010884202D10120BDE8DA
:10054000FC810020FBE786B000273F200090AEA38F
:10055000AEA20A2102A802F031FFAE4908684FF6A8
:10056000FF021040AC4A40F4807010430860AB4872
:100570004FF00009C0F80090A9486FF430510068AE
:100580000844A8490860A84900F5E0500860A74958
:10059000400A0860A64CF8202070FF206070A07010
:1005A00001F00CFB0020964EA24A761C96F904102E
:1005B00052F82120211801F58051135C81F8003890
:1005C000401C6028F6D34FF4E174214640F24910F4
:1005D00001F058FB214640F29F1001F053FB4FF40D
:1005E0008054DFF854A24FF00108307808B1FFF7CB
:1005F00087FE707928B101287ED0307800287CD021
:10060000B2E10A2000F04AFF192221468A48FFF78A
:10061000DAFD022216212046FFF76BFF00286DD07D
:10062000DAF80E10022204F11900FFF762FF002829
:100630007ED09AF80020062A29D2DFE802F02A2A82
:10064000032A2A177D4BDAF80A00596F491C8842A1
:1006500009D25B6F1D1ADAF80E306D1C9D4202D371
:100660001844884215D986F8028012E0DAF80E00A4
:10067000B0F5F42F01D986F80280DAF81200C0F341
:100680000B40B0F5107F04D086F8028001E086F8B8
:100690000280022A01D0052A46D1CDF81490022208
:1006A00004F21D4105A8FFF78EFD0599DAF8040054
:1006B00089B2884201D086F80280CDF814900122D8
:1006C00004F2254105A8FFF77EFD0599BAF801005F
:1006D000C9B2884201D086F802809AF80000022848
:1006E00022D1CDF81490042204F2494105A8FFF765
:1006F0006AFDDAF8120002E059E02EE146E00599C1
:10070000884201D086F80280CDF81490012204F2CC
:100710004D4105A8FFF757FD05999AF80300C9B2A6
:10072000884201D086F802809AF81800401E00E046
:1007300029E0FE2801D286F80280BAF80100A0F56F
:100740007F41FF3901D03F2802D19AF8030028B930
:100750003948FFF7C2FE08B986F80280DAF80E00C1
:100760001B3404443448FFF7B8FE88B14FF480547A
:1007700086F8058086F80390062000F08FFE0A2098
:1007800000F08CFE04E086F8028001E086F802802A
:10079000F078401CC0B2F0700C2801D386F80280BB
:1007A000B07800283FF421AFFFF76DFE1DE7192256
:1007B00021462148FFF707FD9AF81800C0B19AF8C2
:1007C0000000062814D2DFE800F08503055C5E60B7
:1007D00001277FE001279AF8090001287AD1DAF889
:1007E0000A0018B916488069CAF80A00002543E0D3
:1007F00070E00000008009200000094080841E0095
:1008000068000010451B0010460000002573256499
:10081000000000000CED00E00000FA05B000001040
:10082000BC000010A0000010980000109C000010F8
:1008300045010010600000102C010010283B000052
:10084000B03A0000072000F029FEDAF80E00A0EB15
:10085000050BBBF1400F01D94FF0400B6119193165
:100860005A467C48FFF7AFFCDAF80A005A4628449B
:10087000784900F07CFD5D44DAF80E00A842E1D82A
:1008800028E0012726E0012724E001279AF8090043
:1008900003281FD1002519E0072000F0FFFDDAF83A
:1008A0000E00A0EB050BBBF1400F01D94FF0400B40
:1008B000611919315A466748FFF785FC66485A4660
:1008C000006841196348FFF76DFC5D44DAF80E00DB
:1008D000A842E1D89AF8180070B19AF8000058B10F
:1008E0008AF81890192221465C48FFF74CFCC82171
:1008F0004FF47A7001F0C6F9DAF80E001B340444A4
:100900005648FFF7EAFDC8B14FF4805402207071D9
:10091000534880F800900B2000F0C0FD77B100270D
:100920005048816842F2107283685B1A9342FBD38D
:100930004FF42F714FF47A7001F0A4F9F078401C55
:10094000C0B2F0700C2801D386F80280B07800287D
:100950003FF42CAFFFF797FD47E686F8008001F0E3
:1009600030FD012001F0EEFC3D4800780028F3D076
:10097000002102A800F020FC0028EDD04FF48054A4
:1009800086F8059086F803902FE635484FF000086A
:10099000C0F80180A0F80580314FFF207F1C38711E
:1009A00087F8058000F04CFF00F09AFFFFF750FC3D
:1009B00000F038FD002000F071FD01F073FE2A4EBA
:1009C0007069400302D5FFF71FFD48B300240420DF
:1009D00000F064FD7069234D800416D4FFF72BFDF1
:1009E000A0B1FFF728FD88B1FFF725FD70B1042005
:1009F00000F054FD0124A8681C497269920405D4D2
:100A0000AA68121A8A42F8D300E0012444B1A86807
:100A100042F21071AA68121A8A42FBD387F8048046
:100A200000F0DBFC58B1022000F038FD97F904001B
:100A3000401C01D100F0CBFC0120787006E00220C0
:100A400000F02CFD87F8018087F80480FFF78DFB0C
:100A5000FFF779FD451B0010BC0000102C010010B1
:100A600068000010000009400080092080841E00FA
:100A700030B50023FE4A146A2CE0B0F5007F1AD28C
:100A800013280CD014280CD0B0F5FF7F0CD0A0F5A3
:100A90008072FF3A0AD03E280AD9002216E0E2B25C
:100AA00014E0C4F3072211E055220FE0AA220DE062
:100AB000F04A125C0AE0B0F5E05F06D2EE4A02446A
:100AC000A2F5805292F8002E00E00022EB4DEA548D
:100AD000401C5B1C8B42D0D330BD70B5E44D2C6BF9
:100AE000402C00D94024E86AE96902198A4202D9F7
:100AF0000C1A042169702146FFF7BAFF2246DF492C
:100B0000822001F01EFDE86A2044E862286B001B89
:100B10002863DA499F318A68121B8A6008B903206A
:100B200068706878022801D00020087370BD10B585
:100B3000D249D3489F3108600D22822001F001FD87
:100B4000CB490520487010BD70B50E46CD494A69A5
:100B5000520302D5496D490521D4B0F5007F1ED35B
:100B6000C949C34CB0F5E05F1AD28B68A2699A1AE2
:100B7000C64B9A4204D38968A1610021616061611A
:100B80000023BE4CBC4D403407E0C1182944A1F5F8
:100B90008051E25C81F8002E5B1CB342F5D370BD3E
:100BA000626922B98A68A2618A686261A060B84AF3
:100BB0001279002AF3D18A686369D21AB54B9A4236
:100BC0001CD2B54B01221A708A68A26189686161E2
:100BD000A168401A6168884203D9616A884200D2DC
:100BE0006060062000F05AFC61683246BDE8704043
:100BF000A24801F580514030FFF7D4BABDE87040FB
:100C00000C2000F04BBC10B5994CA178E06A42185A
:100C1000E1698A4206D9081AA07005206070022096
:100C200001F04AFCA178E06AFFF78EFFA078E16A44
:100C30000144E162216B091A2163904A9F32936853
:100C4000181A906011B16078052804D10020107343
:100C5000BDE810406BE710BD2DE9F041844CA17850
:100C6000E06A4218E1698A4206D9081AA070052094
:100C70006070022001F020FC0020804DA17805F179
:100C80004003E26A08E016181F5CAE5DBE4202D067
:100C90000020A06202E0401C8842F4D35018E062B9
:100CA000206B401A2063754A9F329368591A9160ED
:100CB00010B16078052808D1A06A20B10020107317
:100CC000BDE8F04133E70120F9E7BDE8F08110B558
:100CD0006A488030017D427CC37C41EA0261827CAB
:100CE000120442EA03221143614A4902D162C17DE2
:100CF000837D41EA032149021163806888420DD057
:100D0000822001F0D9FB022001F0D6FB5B490220D2
:100D10009F310873FFF70BFF002010BD012010BDAD
:100D200070B556480225803000F11F048168002903
:100D30000AD0007B00060CD4022001F0BDFB257315
:100D4000FFF7F5FE002070BD2573FFF7F0FE0020D1
:100D500070BD012070BD10B54848454C803080689A
:100D6000A178884200D2A0704449A2784031822004
:100D700001F0E7FB032060704048A2789F30816853
:100D8000891A81600021017310BD10B53B48803085
:100D90008168002909D0007B000603D5822001F07C
:100DA0008BFB02E0022001F087FB344900209F31D9
:100DB0000873BDE81040BAE610B5FFF7B1FF002890
:100DC0001FD02E4870214030017000214170022256
:100DD0008270C1700171417181710A22C271017208
:100DE00041728172C1723022027301224273817397
:100DF000C173017441741E4912208870BDE810400F
:100E0000A9E710BD1CB5FFF78BFF002868D0234869
:100E10000A22062103886846FFF788F9174800224E
:100E2000403002708023437082700121C170202104
:100E3000017143718271C271412202725422427265
:100E40004F2282724C22C272017341738173C1734B
:100E50004622027450234374722383746923C3743B
:100E60006E230375742343758175C2756C2217E078
:100E70007C000010703A000045010010451B001076
:100E8000555342530080092000000940A08601000C
:100E90006900001020A10700680000100404000091
:100EA000027661224276732282766822C2760177C8
:100EB00041778177C1779DF8011080F820109DF867
:100EC000021080F821109DF8031080F822109DF880
:100ED000041080F82310E84924208870FFF73BFFB6
:100EE0001CBD10B5FFF71CFF00280CD0E348032100
:100EF0000170002141708170C170DF490420887049
:100F0000BDE8104027E710BD10B5FFF709FF002826
:100F100010D0DA4800210170062242708170C17041
:100F2000017141718171C171D34908208870BDE898
:100F3000104010E710BD10B5FFF7F2FE002815D0E5
:100F4000CD4ACE48116A491E0B0E03700B0C43703C
:100F50000B0A8370C17000210171417102238371FA
:100F6000C17108209070BDE81040F4E610BD10B5C6
:100F7000FFF7D6FE002819D0C04800220270427048
:100F800082700821C170BC4B196A0C0E04710C0CE4
:100F900044710C0A8471C171022101724272817222
:100FA000C2720C209870BDE81040D4E610BD2DE947
:100FB000F0410020B04DB14CB04AA978403402E075
:100FC000135C2354401C8842FAD31F2978D121682E
:100FD000AB4881427CD1A94E60685F367060A068E2
:100FE000B060607B4FF0010818B9A07B08B11028F1
:100FF00004D986F80C80BDE8F04198E5E07B1E2816
:10100000F7D00FDC12282ED005DC48B30328F0D12E
:10101000BDE8F041D0E61528EBD01A28E9D1BDE8AB
:10102000F0415EE702272A282DD010DC23281DD0AE
:1010300025281ED02828DCD1FFF749FE00282BD018
:10104000207B000618D56F70BDE8F04145E52F28DC
:101050002AD05528CDD05A28CBD1BDE8F04153E74E
:10106000BDE8F04191E6BDE8F041CBE6BDE8F041D6
:101070007DE7BDE8F0415EE7022001F01DFA37731D
:10108000BDE8F04153E5FFF722FE002804D0207BA5
:10109000000602D485F8018017E6822001F00CFAE0
:1010A0003773BDE8F04142E5FFF711FE0028F3D0A9
:1010B000207B000605D485F80180C5F8288004E669
:1010C00006E0822001F0F8F93773BDE8F0412EE523
:1010D000822001F0F1F9022001F0EEF9062068709B
:1010E000F3E510B564494878022808D003280ED0EB
:1010F00004280FD0052801D10020487010BD5F489A
:101100004030C07B2828F9D1BDE81040E5E4BDE8B7
:1011100010400CE5822001F0CFF9BDE8104006E553
:1011200010B55649022001F0DBF953498870487820
:1011300058B101280CD0022001F0BEF94F4902201D
:101140005F310873BDE81040F1E4BDE810402EE7C0
:101150004A484030C07B2A2804D02F2805D1BDE85A
:10116000104079E5BDE810404DE510BDFFB50246E1
:101170000020002102EB42064FF4405701AD6C46BF
:10118000721845F82120BA4202DD002004B0F0BDFB
:101190003C4B03EB62031B786354D20701D01A095E
:1011A0006254625C02F00F0262548B009A40104459
:1011B000491C0329E4DBE9E7F0B5064600200022DC
:1011C0000023304F4FF4007C52E0521CB45C3CB121
:1011D0009D183D4405F5805595F80058A542F4D07A
:1011E000032A44D303F5C0503A18107F547FD57FAB
:1011F00000EB0420947F240404EB0564204451EAAE
:10120000000401D011B108E00020F0BD1A4949687E
:101210004031884201D90020F0BD002017496C31CF
:101220001C183C4404F5805494F800480C54401CAD
:101230000C28F5D3907ED17E00EB0120117D527DEC
:10124000090401EB026145182846FFF78FFF40F6BD
:10125000F57401E0FFF78AFFC11EA142FAD3A0F5A1
:101260007061FF3901D00020F0BD2846F0BD203369
:101270006345ABD3F0BD00007C000010851B00105F
:10128000555342434501001062B6704730B45E4A80
:101290005D4C032328342360136843F480331360C8
:1012A0005A4A30BC104772B6704770B505460024E4
:1012B0002046FFF7F8FF564B332018605D609960B9
:1012C000DA6054484FF47A710068B0FBF1F01861AD
:1012D00003F114011846FFF7D9FF2046BDE870401E
:1012E000D2E74B4A322313605060916049484FF473
:1012F0007A710068B0FBF1F0D06002F11401104681
:10130000C4E7434A342313605060916041484FF46E
:101310007A710068B0FBF1F0D06002F11401104660
:10132000B4E770B5014600252846FFF7BCFF062448
:10133000394850F824208A4212D93748783850F872
:101340002400884207D121462046FFF7CAFF2146E4
:101350002046FFF7D6FF21462046FFF7C2FF02E0F6
:10136000641C1D2CE5D92846BDE870408CE72DE9AA
:10137000F0412A4C2368002B00D120600020274B2D
:10138000234D5B68283503E01F180E5CEE55401CAA
:101390009042F9D3981860604FF48076B04213D130
:1013A0002068FFF7BEFF1A4D1435286800B1FEE72C
:1013B0001749324628312068FFF777FF286800B1C7
:1013C000FEE70020606020600020BDE8F081144945
:1013D0004FF4C0400860FEF78FBE002146F2044083
:1013E0000088A0F51942993A0AD04FF4C0404FF452
:1013F000002304C811449842FBD319B10020704760
:10140000012070470120704788C10F40F11FFF1F66
:10141000001C0010D8000010283B0000C000001085
:1014200008ED00E0002070478449C20702D04FF069
:1014300000728A67800702D54FF0806088670020BD
:1014400070477E49C20702D04FF00072CA6780071A
:1014500002D54FF08060C867002070470021774AAE
:10146000C30703D0536F9B0100D50121800704D52A
:10147000506F400101D541F0020188B2704710B5AC
:1014800004462046FFF7EAFF03461846FFF7D9FF58
:1014900024EA0300FFF7C8FF002010BDF0B50346A3
:1014A000674C002B0AD06068042503270226052814
:1014B00007D2DFE800F0072B5C8DB80000206060E9
:1014C000A060F0BD042B02D0052B07D009E003205B
:1014D000FFF7B7FF0120FFF7A7FF02E00120FFF7AA
:1014E000B0FF0125022B09D0012BEAD10320FFF721
:1014F000A8FF0120FFF798FF6560F0BD0320FFF70C
:10150000A0FF0220FFF790FF6560F0BD062B10D012
:10151000032B16D00A2B1CD0092B1AD00D2B1FD051
:101520000C2BF2D10320FFF78CFFBDE8F040012027
:101530007AE70320FFF785FF0220FFF775FF66605B
:10154000F0BD0320FFF77DFF0120FFF76DFF67600F
:10155000F0BD0320FFF775FFBDE8F040022063E710
:101560000320FFF76EFFBDE8F04002205CE7062B8A
:101570000ED00A2B15D0092B1BD00C2B21D00D2BF4
:10158000E6D10320FFF75DFFBDE8F04002204BE706
:10159000A068411CA160C006DAD1BDE8F04002207D
:1015A0006DE70320FFF74DFF0220FFF73DFF676067
:1015B000F0BD0320FFF745FF0120FFF735FF656011
:1015C000F0BD0320FFF73DFFBDE8F04001202BE711
:1015D000072B0DD00A2B17D00B2B1CD0092BEFD1CA
:1015E0000320FFF72EFF0120FFF71EFF6560F0BD0F
:1015F0000220FFF726FFA068411CA1608006F6D1FB
:10160000BDE8F04001203AE70320FFF71AFFBDE8EC
:10161000F040012008E70320FFF713FF0220FFF747
:1016200003FF6560F0BD062BFCD10320FFF709FF27
:101630000220FFF7F9FE6660F0BD0000008009207F
:10164000CC000010F0B5A14DD5F804014FF0000218
:10165000C1059F4852D4D5F80C119E4BC90707D03D
:10166000D5F8A011490626D40260426082609EE04F
:10167000D5F80411C9061AD0D5F8041101F01F01DC
:10168000B3FBF1F10160D5F8A841E40611D0D5F81B
:10169000A84104F01F04B3FBF4F34360D5F8003114
:1016A00003F001035B1CB1FBF3F181607FE00021DB
:1016B000E8E70023F1E7D5F80411C9061AD0D5F8F8
:1016C000041101F01F01B3FBF1F10160D5F8A8414D
:1016D000E40611D0D5F8A84104F01F04B3FBF4F3DD
:1016E0004360D5F8003103F001035B1CB1FBF3F15B
:1016F00081605CE00021E8E70023F1E7D5F888107D
:10170000C90503D402604260826050E0D5F80C1134
:10171000C90707D0D5F8A011490628D40260426055
:10172000826044E055F8881F01F01F035B1CE96FDD
:1017300001F01F01D5F8204104F01F04AE6F883D71
:1017400006F00106761C71B1624F5F43B7FBF1F101
:10175000016054B15F4F7B43B3FBF4F34360B1FBD3
:10176000F6F1816023E00021F2E70023F6E755F867
:10177000881F01F01F035B1CE96F01F01F01D5F802
:10178000204104F01F04AE6F883D06F00106761C70
:10179000E1B1504F5F43B7FBF1F10160C4B14D4F70
:1017A0007B43B3FBF4F34360B1FBF6F18160D5F802
:1017B0000811C90528D5D5F8081111F01F0109D065
:1017C000042909D0062907D0C260F0BD0021E4E752
:1017D0000023E8E7C260F0BD903555F8081C01F021
:1017E0001F01491CAA6F02F01F02EB6FDB0705D037
:1017F000384B5943B1FBF2F1C160F0BD354B594351
:10180000B1FBF2F1C160F0BDD5F80811890515D51D
:10181000D5F80C11C90708D0D5F8A8102D4A01F049
:101820001F01491C5143C160F0BDD5F88810294AF9
:1018300001F01F01491C5143C160F0BDC260F0BD01
:1018400010B422482021C0F8A011D0F8A0114906F8
:10185000FBD501228030C0F88C2009214160026054
:10186000AA24C4605523C3608038D0F88810490585
:10187000FBD52321A03041600260C460C360A03862
:10188000D0F8A8104905FBD58C3040F201118167D2
:1018900040F20121C16742670221C0F828110421EA
:1018A000C0F81C110C4981630021C0F83C11D0F82C
:1018B000242142F00302C0F8242145F23A0240F804
:1018C0008C2C0648016010BCBCE6000000C00F4034
:1018D000D8000010001BB700FE9FF8F708ED00E0ED
:1018E000F0B5B049032008630020C1F80801AE48F4
:1018F00004228265026C42F004020264AB4A8A66EA
:1019000000220A611022C261026822F01002026005
:101910000322C1F87022C1F8742200224A644FF4F5
:1019200000328261026842F4003202600922C1F88A
:101930000021C1F804211022C1F8D420520482638E
:10194000026A42F4001202620D22C1F8D020C1F8EE
:10195000E0200022C1F8F4204FF00052C263026A76
:1019600042F0005202620022C1F8F0204FF0805293
:10197000C263026A42F0805202621022CA67020405
:101980008261026842F0004202601022C1F8142114
:1019900020278765026C42F0200202641022C1F801
:1019A0001C218022C265026C22F080020264902613
:1019B000C1F8FC600204C263026A22F000420262C3
:1019C0001022C1F8DC20D204C263026A22F40002B1
:1019D000026201230B660122CA654A660322C1F82E
:1019E000D8200522C1F8E42001228A601122CA60B1
:1019F0000124CC630A640224C1F820411225C1F8F5
:101A000024510C604D600C604D6010248C659C0569
:101A1000C461046844F4800404600124CC630A6453
:101A20001022C1F82C21CA14C265026C42F4006273
:101A300002641022C1F830218A14C265026C42F49B
:101A40008052026440F282224A629A240C62CA6185
:101A500010224A618761026842F02002026010226F
:101A60008A6140258561026842F0400202600122DD
:101A70000A67CA6640F20242CA628A621022C1F84C
:101A8000E82092058263046A44F0806404621024B2
:101A9000C1F8EC405400C463046A24F0006404629A
:101AA0004E635413C461046824F400540460002499
:101AB000C1F8E841C267026E42F08062026600220D
:101AC000C1F8E4215A06C267026E42F00072026653
:101AD0008A22C1F8F8200822C1F8C820D403C463C0
:101AE000066A46F4802606621026C1F828610E15A3
:101AF000C665066C26F4806606640126C1F880601F
:101B0000C1F88460C1F89060C1F8A060C1F8A46019
:101B1000C1F8A860C1F8B860C1F8BC60C1F8C06085
:101B2000C1F8C4600026C1F81861C565056C45F0B0
:101B3000400505640A655504C561056825F48015EE
:101B40000560CA641504C561056825F400250560B3
:101B50008A64C461046824F4802404600024C1F809
:101B60000C418265026C42F0080202640022C1F856
:101B7000102110228265026C42F0100202640C48AF
:101B80000C4A0068904204D141F8B83F8B60CB60AA
:101B9000F0BD094A9042FBD1812041F8B80F88601E
:101BA000C860F0BD00C002400080092002000100B2
:101BB000C8000010473F1927473F19474E490020EA
:101BC0000867C86002224A6188613022CA634B49B3
:101BD0008A684B490A6048604A4908604A49086077
:101BE00078464A490860002070472DE9F04341F2E9
:101BF00088320023434C444D444E904208D8642818
:101C000000D228B942F21072914201D8052907D2B8
:101C1000862020602B60784630608620BDE8F08307
:101C2000DFF8D8C0DCF80820354FD7F80080A2EBE9
:101C300008087A6802EB4209C9EBC212B8EBC20F7E
:101C400006D2052020602B60784630600520E5E74D
:101C5000294A4FF00208C2F8048048B1DFF8B0907A
:101C6000B9FBF0F040109061C2F804800120506090
:101C7000DCF808003860796023602B6078463060BB
:101C80000020CBE7F0B50C461D4D00266E602146C6
:101C9000FFF7ABFF1B4F000601D53868F0BD04EB22
:101CA0004400C0EBC411154A286893681B1AB3EBB3
:101CB000C10FFAD3104802214160C16B01F0FE014F
:101CC000C1636E603868F0BD0C4880680C490A68D2
:101CD000821A486800EB4003C3EBC010B2EBC00FA0
:101CE00008D3054802224260C26B02F0FE02C263C2
:101CF000002048607047000000800040000009405C
:101D0000EC0000107000001074000010780000104B
:101D100080C3C901FC4800218180017041704FF0EF
:101D200001128260C1607047F7491C31002000F049
:101D3000D7BB10B5F44C1434A288402A00D94022F5
:101D40008020216800F0FDFB216801442160A1880A
:101D5000081AA08010BD10B5EB4C00201434216887
:101D600000F0BEFB216801442160A188081AA08010
:101D700010BD00221146802000F0E3BBE3490020A3
:101D800000F0AEBB70B5E048DF4C1C3004F1140429
:101D9000007810F01F000BD0DB4BDC4D03F11C0171
:101DA0005A780979012809D0022813D0002070BD83
:101DB000D548001D2060FFF7BCFF27E042B19878AE
:101DC000814205D2002028802560FFF7B2FF1DE088
:101DD000002070BD01F08F00010605D500F00F0650
:101DE0004FF48031B14001E0012181400AB9000780
:101DF0000ED1986808420BD0D868084201D0012063
:101E000000E0002028802560FFF793FF012070BDCF
:101E1000002070BD70B50246BB4BBB4D1C3319464C
:101E20001878498810F01F0005D0012818D0022822
:101E300018D0002070BD012901D0002070BD3AB13A
:101E4000012000F0E7FAA88840F00200A8802CE00A
:101E5000002000F0DFFAA88820F00200A88024E02B
:101E6000002070BD187900F08F00030605D500F042
:101E70000F034FF480349C4001E0012484406B78D0
:101E8000ABB1030713D0AB68234210D009B10020D7
:101E900070BD2AB100F010FBE8682043E86004E060
:101EA00000F014FBE868A043E860012070BD00204A
:101EB00070BD10B594481C30007810F01F01924896
:101EC00000F11C00C07803D001292FD0002010BDE4
:101ED0008D4B1433012808D003F1080102288A78B9
:101EE00007D0032816D0002010BD894818601220A2
:101EF00014E08848002104E004780CB144882044B0
:101F0000491C8A42F8D1017811B11860408805E077
:101F1000002010BD804810441860007899888142E4
:101F200000D99880FFF705FF012010BD002010BDEB
:101F30002DE9F05F0027DFF8D0B1734E0BF11C0BD9
:101F4000B8469BF802004FF001094FF4803A002890
:101F500068D0704C62E06078022804D0042840D039
:101F6000052859D13FE061799BF80200814235D1C3
:101F700070702079B07000206349103101F8008042
:101F8000401C0428FAD30125B16809FA05F008427B
:101F900002D0284600F07CFAB1680AFA05F008423F
:101FA00003D045F0800000F073FA6D1C102DEBD3C8
:101FB0004FF001103546B060C5F80C80012000F0EC
:101FC0002AFAE079400604D5A88840F00100A880EC
:101FD00022E0A88820F00100A8801DE06088044469
:101FE0001CE0E77818E0BFB9A07800F08F0528065C
:101FF00004D505F00F000AFA00F001E009FA05F037
:10200000B1680143B160204600F01DFA284600F097
:1020100035FA284600F046FA207804442078002853
:1020200099D11EE086F801800124B16809FA04F014
:10203000084202D0204600F02BFAB1680AFA04F0F8
:10204000084203D044F0800000F022FA641C102CF7
:10205000EBD34FF00110B060C6F80C80002000F008
:10206000DAF99BF802007178884202D10120BDE8BC
:10207000F09F0020FBE72DE9F84F00270026B2462D
:10208000B146DFF884B09BF80100002803D000209F
:102090000090204C72E00020BDE8F88F60780228A4
:1020A00004D004280AD0052866D11BE060799BF88B
:1020B0000110884260D0608804445FE0A778E67829
:1020C0004FF0000910481C300179B94254D1807892
:1020D000B04251D1012000900B48103010F807A0F9
:1020E000C65549E008481C300179B94244D1A1786D
:1020F00001F08F085FEA086110D508F00F014FF476
:1021000080358D400DE00000F4000010281D001007
:10211000A03B0000B23B0000D33B0000012505FAC4
:1021200008F58078B04215D1DBF808002843CBF8D9
:102130000800DBF80C00A843CBF80C00204600F0A8
:1021400082F9404600F09AF9404600F0ABF949EABE
:10215000050911E056450FD119EA050F0CD1DBF83E
:102160000800A843CBF80800DBF80C00A843CBF824
:102170000C00404600F08CF92078044420780028B8
:102180008CD1009888E72DE9F041544F0026A7F143
:1021900008053978A5F1140408281FD2DFE800F0FB
:1021A0001E0477851E1E9994FFF7BEFD3878C0097E
:1021B00000F063F9F888A8803878C0F3411181BB3A
:1021C00079780C295ED2DFE801F0060B5D125D190B
:1021D00023272D364253FFF7D5FD10B3BDE8F0811C
:1021E0000020FFF717FEE0B1BDE8F041C1E5012096
:1021F000FFF710FEA8B1BDE8F041BAE510F01F0FDF
:1022000040D1B87840F080002070BDE8F041B0E5E2
:10221000FFF74FFE28B1E1E7002000F04DF9AE8056
:10222000DCE72FE010F01F0F2CD12C481B38286062
:10223000BDE8F0417DE510F01F0F23D1FFF778FED8
:1022400000B3FFF796FDBDE8F041FEF7ABB800F034
:102250001F00012816D16078A0B13879A178884292
:1022600010D21E490C3908442860BDE8F04160E5F1
:1022700000F01F00012805D1FFF7FDFE10B1BDE8F9
:10228000F04176E5802000F017F9AE80A6E7080659
:1022900008D4A8880028A1D0FFF75DFDA8880028F1
:1022A000F0D09BE7BDE8F04168E5080602D5BDE83F
:1022B000F0413EE52078010690D500F07F002070C7
:1022C000BDE8F04100F054B8BDE8F041802000F0D6
:1022D000FDB8BDE8F041002000F0F8B81001001092
:1022E00001460807C00E090600D5401C7047DB49AF
:1022F0001022C1F80822C1F81002D1F80002C0066D
:10230000FBD57047D54A1023C2F80832C2F8100234
:10231000D2F80002C006FBD5C2F80832C2F810128B
:10232000D2F80002C006FBD57047CC493022C1F874
:102330000822C1F81002D1F800028006FBD5D1F8BE
:102340001402704710B50446002C01D0012100E0B2
:1023500000214FF4807040EA0141C148FFF7D2FFED
:10236000C0484FF480210CB1816310BDC16310BD22
:1023700030B540F080014FF4807040EA0141BA4D21
:102380000C462846FFF7BEFF21462846BDE83040F0
:10239000B8E7B64800210160402141600122026097
:1023A0004160A0F51270D0F80012C905FBD500F508
:1023B00001704FF0FF314163016341600C21016006
:1023C000704730B5AA4C1A232360211D0A6833EAEE
:1023D0000200FBD1A748012242678267A64D002276
:1023E0002A608A22C0F8F82023600A6833EA0200D3
:1023F000FBD1A2494FF08070C1F8FC01A04B202214
:102400001A70C867FFF7C5FFBDE830400020AFE78E
:1024100070477047704710B5002801D0012000E0D8
:1024200000204FF4807444EA00419648FFF76AFFA9
:102430008A480321C0F84412D0F80012C905FBD520
:10244000C0F8084210BD10B502469078FFF748FF6B
:102450008649091F0B680124844023430B604860B0
:1024600090888860A1F51171D1F80002C005FBD5F4
:102470004FF48070C1F8080210BD704700B5FFF737
:102480002FFF81495DF804EB41EA0040891339E7E9
:1024900000B5FFF725FF7C495DF804EB41EA0040F9
:1024A0007A492FE700B5FFF71BFF77495DF804EB8A
:1024B00041EA0040891325E700B5FFF711FF724993
:1024C0005DF804EB41EA004071491BE700B5FFF7F6
:1024D00007FF6D495DF804EB41EA0040891311E7FD
:1024E00070B506465D4B06F00F00012202EB80003E
:1024F000C3F82802D3F820020205FBD5C0F3090572
:102500000022EC1C04E0D3F8180241F8040B521C22
:10251000B2EB940FF7D30020C3F8280241F2482011
:10252000F040C0070BD13046FFF7DAFE4FF4A06150
:1025300041EA0040FFF7DBFE5648FFF7D8FE284689
:1025400070BD70B51646454D00F00F02022303EB37
:102550008202C5F82822C5F824620023F41C04E096
:1025600051F8042BC5F81C225B1CB3EB940FF7D376
:102570000021C5F82812FFF7B3FE4FF4A06141EA2D
:102580000040FFF7B4FE4448FFF7B1FE304670BD8F
:102590002DE9F041314FD7F80032C7F8083218075B
:1025A00025D52F48FFF7A3FE3C48FFF7BEFEC10626
:1025B00005D5FFF7EEFEBDE8F041FDF7E4BE81076B
:1025C00005D5BDE8F04100F00100FDF7D6BE0107DA
:1025D0000DD5400705D5FFF71BFFBDE8F041FDF71E
:1025E000D9BEFFF716FFBDE8F041FDF7DABE580788
:1025F00021D54FF001082A4E19E00024D7F8300207
:1026000008FA04F528420FD06008C7F83852D7F806
:1026100000128906FBD5D7F81412E2070DD056F840
:10262000201009B103208847641C202CE6D3D7F87A
:1026300030020028E1D1BDE8F0813CB9490705D559
:10264000316819B1316801208847EDE756F820104C
:102650000029E9D002208847E6E7000000C00820F2
:102660000005FE00008009200005D00048C20820B7
:10267000F4CF082000C0024010C1082084E000E030
:1026800018E400E00005D80000054000000120002B
:10269000000101000005F2000005FA000002FE0042
:1026A000443C000019480621016107210160002116
:1026B0004161416202214160C168C906FCD400E069
:1026C0008168C1684907FBD4002070470F498860C2
:1026D000C868C006FCD48868704700B502460B463F
:1026E00003E012F8010BFFF7F1FF5B1E581CF8D155
:1026F00000BD00B502460B4604E00020FFF7E6FFF0
:1027000002F8010B5B1E581CF7D100BD000003400E
:102710002DE9F0478146F84E4FF08077402430682D
:10272000F64DB84249D100BF00BF00BF00BF00BF97
:1027300000BF00BF00BF00BF00BF00BF00BF00BFA1
:1027400000BF00BF00BF00BF00BF00BF00BF00BF91
:1027500000BF00BF00BF00BF00BF00BF00BF00BF81
:1027600000BF00BF00BFEC611520FFF7AFFF0020E6
:10277000FFF7ACFF00F0FF08AC6100BF00BF00BF77
:1027800000BF00BF00BF00BF00BF00BF00BF00BF51
:1027900000BF00BF00BF00BF00BF00BF00BF00BF41
:1027A00000BF00BF00BF00BF00BF00BF00BF00BF31
:1027B00000BF00BF00BF00BF00BF00BF00BF00BF21
:1027C00000BF00BF00BF00BF00BF00BF00BF00BF11
:1027D00000BF00BF00BF00BF00BF00BF00BF00BF01
:1027E00000BF00BF00BF00BF00BF00BF00BF00BFF1
:1027F00000BF00BF00BF00BF00BFEC610620FFF7B5
:1028000065FFAC6100BF00BF00BF00BF00BF00BFDD
:1028100000BF00BF00BF00BF00BF00BF00BF00BFC0
:1028200000BF00BF00BF00BF00BF00BF00BF00BFB0
:1028300000BF00BF00BF00BF00BF00BF00BF00BFA0
:1028400000BF00BF00BF00BF00BF00BF00BF00BF90
:1028500000BF00BF00BF00BF00BF00BF00BF00BF80
:1028600000BF00BF00BF00BF00BF00BF00BF00BF70
:1028700000BF00BF00BF00BF00BF00BF00BF00BF60
:1028800000BF00BFEC610120FFF720FF4FEA890085
:10289000FFF71CFF3068B84202D14046FFF716FF31
:1028A000AC6100BF00BF00BF00BF00BF00BF00BFE2
:1028B00000BF00BF00BF00BF00BF00BF00BF00BF20
:1028C00000BF00BF00BF00BF00BF00BF00BF00BF10
:1028D00000BF00BF00BF00BF00BF00BF00BF00BF00
:1028E00000BFBDE8F0872DE9F8430025009500BF43
:1028F00000BF00BF00BF00BF00BF00BF00BF00BFE0
:1029000000BF00BF00BF00BF00BF00BF00BF00BFCF
:1029100000BF00BF00BF00BF00BF00BF00BF00BFBF
:1029200000BF00BF00BF00BF00BF00BF00BF402608
:10293000724FFE619F20FFF7C9FE0020FFF7C6FE21
:10294000C4B28DF800400020FFF7C0FE00F0FF0980
:102950008DF801900020FFF7B9FEC0B28DF802009B
:10296000BE6100BF00BF00BF00BF00BF00BF00BF0F
:1029700000BF00BF00BF00BF00BF00BF00BF00BF5F
:1029800000BF00BF00BF00BF00BF00BF00BF00BF4F
:1029900000BF00BF00BF00BF00BF00BF00BF00BF3F
:1029A00000BF574E574FDFF86081C22C02D1B9F1FA
:1029B000200F09D082203060212038607846C8F886
:1029C00000008220BDE8F8834B49142810D0152858
:1029D00012D0162814D0182816D00D600020FFF74A
:1029E00097FE35603D607846C8F800000020E9E7B2
:1029F0004FF480100860F1E74FF400100860EDE735
:102A00004FF480000860E9E74FF080700860E5E768
:102A10002DE9F04F89B00D46DDF8489092461F46EB
:102A20000024DFF8DC80B9F1000F4ED04FF480565F
:102A30000146324601A8FDF73BFCDDE90101CDE985
:102A400005013246691C01A8FDF732FCDDE90101F0
:102A5000CDE903013246514601A8FDF729FCDDE925
:102A60000101CDE90701A346A9EB04050898C0F5CB
:102A70008050A84200D20546089838B105990798B9
:102A8000884279D1069908988842FAD14FF480504B
:102A900000F0B8FD0646300022D00599079888421C
:102AA0006BD10699089888427ED1DDE907020003C0
:102AB000314600F097F9000628D5304600F07AFD3F
:102AC000D8F8000009B0BDE8F08F8620C8F80000F3
:102AD0000C480921016079460B4801608620F1E726
:102AE0008220C8F800000748222101607946064884
:102AF00001608220E6E7000020010010008009202C
:102B000070000010740000107800001003990798FE
:102B1000884211D1DDE9031000EB01300499C1F5C1
:102B20008052314400F05EF9000605D5304600F0D1
:102B300041FDD8F80000C5E7079800F0D8F9000675
:102B400005D5304600F036FDD8F80000BAE7089801
:102B5000391930442A46FDF7B5FB08983146421929
:102B60000798000300F0ABFB000607D5304600F0E5
:102B700021FDD8F80000A5E75FE015E0039907986C
:102B8000884256D1DDE9031000EB01300499C1F50C
:102B90008052314400F093FB00064AD5304600F0E5
:102BA00009FDD8F800008DE703990798884211D1F4
:102BB000DDE9031000EB01300499C1F58052314684
:102BC00000F010F9000605D5304600F0F3FCD8F807
:102BD000000077E7079800F08AF9000605D530462F
:102BE00000F0E8FCD8F800006CE739190AEB0400A3
:102BF0002A4600F064FB000605D5304600F0DAFCFA
:102C0000D8F800005EE703990798884211D1DDE902
:102C1000031000EB01300499C1F58052314600F0F9
:102C20004EFB000605D5304600F0C4FCD8F8000085
:102C300048E7304600F0BEFC0AE039190AEB040010
:102C40002A4600F03CFB000602D5D8F8000039E720
:102C50002C440798401C0790CDF820B04C45FFF459
:102C600003AFC8F800B00548C0F800B07946044882
:102C70000160002026E703480068704774000010D8
:102C8000780000102001001070B5044600BF00BF9E
:102C900000BF00BF00BF00BF00BF00BF00BF00BF3C
:102CA00000BF00BF00BF00BF00BF00BF00BF00BF2C
:102CB00000BF00BF00BF00BF00BF00BF00BF00BF1C
:102CC00000BF00BF00BF00BF00BF00BF4026D24D05
:102CD000EE610520FFF7FAFC0020FFF7F7FC2070FB
:102CE000AE6100BF00BF00BF00BF00BF00BF00BF9C
:102CF00000BF00BF00BF00BF00BF00BF00BF00BFDC
:102D000000BF00BF00BF00BF00BF00BF00BF00BFCB
:102D100000BF00BF00BF00BF00BF00BF00BF00BFBB
:102D200000BF207800F0010070BD2DE9F04106469B
:102D30000F46BA4CA56806E0A068401BB04202D31B
:102D40000120BDE8F0813846FFF79EFF0028F3D14F
:102D5000F7E770B500BF00BF00BF00BF00BF00BFF6
:102D600000BF00BF00BF00BF00BF00BF00BF00BF6B
:102D700000BF00BF00BF00BF00BF00BF00BF00BF5B
:102D800000BF00BF00BF00BF00BF00BF00BF00BF4B
:102D900000BF00BF4025A04CE5610620FFF796FC70
:102DA000A56100BF00BF00BF00BF00BF00BF00BFE4
:102DB00000BF00BF00BF00BF00BF00BF00BF00BF1B
:102DC00000BF00BF00BF00BF00BF00BF00BF00BF0B
:102DD00000BF00BF00BF00BF00BF00BF00BF00BFFB
:102DE00000BF70BD2DE9FC5F04468A4691468C4DBC
:102DF0008C4E8D4F4FF00008B9F1000F0DD001A996
:102E00008A48FFF792FF80B182202860212030603D
:102E1000784638608220BDE8FC9FC5F80080C6F87F
:102E20000080784638600020F5E703208DF8000028
:102E3000200C8DF80100200A8DF802008DF8034067
:102E400000BF00BF00BF00BF00BF00BF00BF00BF8A
:102E500000BF00BF00BF00BF00BF00BF00BF00BF7A
:102E600000BF00BF00BF00BF00BF00BF00BF00BF6A
:102E700000BF00BF00BF00BF00BF00BF00BF00BF5A
:102E80004024DFF894B1CBF81C4004216846FFF7DA
:102E900024FC49465046FFF72CFCCBF8184000BFF5
:102EA00000BF00BF00BF00BF00BF00BF00BF00BF2A
:102EB00000BF00BF00BF00BF00BF00BF00BF00BF1A
:102EC00000BF00BF00BF00BF00BF00BF00BF00BF0A
:102ED00000BF00BF00BF00BF00BF00BF00BFC5F8FC
:102EE0000080C6F8008078463860002093E72DE91E
:102EF000FC47044601A94D48FFF717FF484FDFF88C
:102F00002481DFF8249150B1822038602220C8F853
:102F100000007846C9F800008220BDE8FC879DF8D3
:102F20000400800701D4FFF714FF20208DF8000073
:102F300020098DF8010020018DF8020000248DF891
:102F4000034000BF00BF00BF00BF00BF00BF00BF05
:102F500000BF00BF00BF00BF00BF00BF00BF00BF79
:102F600000BF00BF00BF00BF00BF00BF00BF00BF69
:102F700000BF00BF00BF00BF00BF00BF00BF00BF59
:102F800000BF4026244DEE6104216846FFF7A5FBF3
:102F9000AE6100BF00BF00BF00BF00BF00BF00BFE9
:102FA00000BF00BF00BF00BF00BF00BF00BF00BF29
:102FB00000BF00BF00BF00BF00BF00BF00BF00BF19
:102FC00000BF00BF00BF00BF00BF00BF00BF00BF09
:102FD00000BF3C60C8F800407846C9F800000020F7
:102FE0009BE770B50F4D104E0D4C002A05D0FFF732
:102FF000F9FE000609D5206870BD862020600920F2
:10300000286078463060862070BD002020602860EF
:1030100078463060002070BD008009200000094023
:10302000700000107400001078000010A0860100ED
:1030300070B5044600BF00BF00BF00BF00BF00BFA7
:1030400000BF00BF00BF00BF00BF00BF00BF00BF88
:1030500000BF00BF00BF00BF00BF00BF00BF00BF78
:1030600000BF00BF00BF00BF00BF00BF00BF00BF68
:1030700000BF00BF4026A94DEE610520FFF726FBEB
:103080000020FFF723FB2070AE6100BF00BF00BF30
:1030900000BF00BF00BF00BF00BF00BF00BF00BF38
:1030A00000BF00BF00BF00BF00BF00BF00BF00BF28
:1030B00000BF00BF00BF00BF00BF00BF00BF00BF18
:1030C00000BF00BF00BF00BF00BF207800F00100BC
:1030D00070BD2DE9F04106460F46914CA56806E00B
:1030E000A068401BB04202D30120BDE8F081384601
:1030F000FFF79EFF0028F3D1F7E72DE9F34F85B0E6
:10310000044604A98748FFF7E4FF874D874E884FA0
:103110004FF0820A48B1C5F800A0212030607846FF
:103120003860822007B0BDE8F08FFFF712FE422022
:103130008DF804004FF0000BCDF805B0CDF809B0C4
:10314000ADF80DB000BF00BF00BF00BF00BF00BFA3
:1031500000BF00BF00BF00BF00BF00BF00BF00BF77
:1031600000BF00BF00BF00BF00BF00BF00BF00BF67
:1031700000BF00BF00BF00BF00BF00BF00BF00BF57
:1031800000BF00BFDFF894814FF04009C8F81C90E1
:103190000B2101A8FFF7A1FAC8F8189000BF00BFE3
:1031A00000BF00BF00BF00BF00BF00BF00BF00BF27
:1031B00000BF00BF00BF00BF00BF00BF00BF00BF17
:1031C00000BF00BF00BF00BF00BF00BF00BF00BF07
:1031D00000BF00BF00BF00BF00BF00BF04A951482F
:1031E000FFF777FF38B1C5F800A02220306078469D
:1031F0003860822096E79DF81000800701D4FFF721
:10320000A8FD02208DF80400200C8DF80500200A8E
:103210008DF806008DF8074006988DF8080000BF6D
:1032200000BF00BF00BF00BF00BF00BF00BF00BFA6
:1032300000BF00BF00BF00BF00BF00BF00BF00BF96
:1032400000BF00BF00BF00BF00BF00BF00BF00BF86
:1032500000BF00BF00BF00BF00BF00BF00BFC8F875
:103260001C90052101A8FFF738FAC8F8189000BF94
:1032700000BF00BF00BF00BF00BF00BF00BF00BF56
:1032800000BF00BF00BF00BF00BF00BF00BF00BF46
:1032900000BF00BF00BF00BF00BF00BF00BF00BF36
:1032A00000BF00BF00BF00BF00BF00BF00BFC5F828
:1032B00000B0C6F800B078463860002032E72DE94B
:1032C000F05F80460D461646174FDFF860A0DFF826
:1032D00060B04FF00009002E01D0002413E0C7F8C1
:1032E0000090CAF800907846CBF800000020BDE8B6
:1032F000F09F295D08EB0400FFF7FFFE000601D5F3
:103300003868F4E7641CB442F3D3C7F80090CAF8F5
:1033100000907846CBF800000020E8E70080092004
:1033200000000940A0860100700000107400001029
:103330007800001070B500242546002801DA012429
:103340004042002901DA01254942FDF73FF8AC422D
:1033500000D04042002C00D0494270BD064C074DC1
:1033600006E0E06840F0010394E807009847103455
:10337000AC42F6D3FCF7BAFE843C0000A43C00004B
:1033800030B58C1810F8012B12F00F0301D110F892
:10339000013B120906D110F8012B03E010F8015B84
:1033A00001F8015B5B1EF9D101E001F8013B521EFF
:1033B000FBD1A142E6D3002030BD00000FB41CB504
:1033C0000A46521ECDE9000207A9054B6A46069837
:1033D00000F008F8009A002111701CBC5DF814FB85
:1033E0009D3500002DE9FF4F8BB09A460F460546EC
:1033F000002606E025280BD052460D9990476D1CFB
:10340000761C28780028F5D10FB03046BDE8F08F43
:103410000024A0460122604900E0044315F8013F62
:10342000203B02FA03F00842F7D128782E2817D162
:1034300015F8010F44F004042A280ED06FF02F0273
:103440002878A0F1300109290AD808EB880102EB9D
:10345000410100EB01086D1CF2E757F8048B6D1C6D
:10346000287869283ED006DC0028CDD063280BD010
:10347000642804D136E0732810D075284BD052460A
:103480000D999047761C85E017F8040B8DF8000025
:1034900000208DF80100E946012003E057F8049B65
:1034A0004FF0FF3061074FF0000401D40AE0641CC4
:1034B00044450DDA8442FADB19F804100029F6D1EC
:1034C00006E0641C8442FCDB19F804100029F8D1E2
:1034D000264404E019F8010B52460D999047641EEA
:1034E000F8D257E001CF4FF00A0B002802DA404231
:1034F0002D2102E0210504D52B218DF82410012176
:1035000003E0E10705D02021F7E70DF1200908913C
:103510000CE00021F9E701CF4FF00A0BF9E759461B
:10352000FCF754FF01F1300209F8012D0028F6D113
:10353000ADEB090000F1200B600701D44FF001084A
:10354000D84502DDA8EB0B0000E0002080460024F7
:1035500006E009A85246005D0D999047641C761C50
:1035600008988442F5DB04E0302052460D999047DC
:10357000761CB8F10001A8F10108F5DC05E019F8A6
:10358000010B52460D999047761CBBF10001ABF13F
:10359000010BF4DC6D1C34E7092801004A68002A9D
:1035A00006D00A68531C0B6010704868401E4860C3
:1035B0007047000010B5002821D0114B0022001FD9
:1035C000196803E0814203D80A4649680029F9D105
:1035D00052B11368841A9C4204D1006818441060E8
:1035E000104602E0506000E0186039B102680B1A22
:1035F000934203D10B681A4402604968416010BDD0
:1036000024010010F0B50B30154D20F00701002407
:10361000144A0FE003688B420BD38B4205D95E1A24
:1036200043184768C3E9006700E04368136002C0BD
:1036300004E0021D10680028ECD12046002802D1C9
:10364000286808B10020F0BD064A07481060074A04
:10365000121A22F00702C0E9002401202860D7E7EF
:1036600028010010240100106C1D0010688D00104E
:1036700000050F0A1B1E141133363C39282D272252
:1036800063666C69787D777250555F5A4B4E444142
:10369000C3C6CCC9D8DDD7D2F0F5FFFAEBEEE4E132
:1036A000A0A5AFAABBBEB4B193969C99888D878222
:1036B00083868C89989D9792B0B5BFBAABAEA4A112
:1036C000E0E5EFEAFBFEF4F1D3D6DCD9C8CDC7C202
:1036D00040454F4A5B5E545173767C79686D6762F2
:1036E00023262C29383D373210151F1A0B0E0401E2
:1036F00003060C09181D171230353F3A2B2E2421D2
:1037000060656F6A7B7E747153565C59484D4742C1
:10371000C0C5CFCADBDED4D1F3F6FCF9E8EDE7E2B1
:10372000A3A6ACA9B8BDB7B290959F9A8B8E8481A1
:1037300080858F8A9B9E9491B3B6BCB9A8ADA7A291
:10374000E3E6ECE9F8FDF7F2D0D5DFDACBCEC4C181
:1037500043464C49585D575270757F7A6B6E646171
:1037600020252F2A3B3E343113161C19080D070261
:1037700000002110422063308440A550C660E770ED
:10378000088129914AA16BB18CC1ADD1CEE1EFF195
:103790003112100273325222B5529442F772D6623D
:1037A000399318837BB35AA3BDD39CC3FFF3DEE3E5
:1037B0006224433420040114E664C774A44485548D
:1037C0006AA54BB528850995EEE5CFF5ACC58DD535
:1037D0005336722611163006D776F6669556B446DD
:1037E0005BB77AA719973887DFF7FEE79DD7BCC785
:1037F000C448E5588668A77840086118022823382D
:10380000CCC9EDD98EE9AFF9488969990AA92BB9D4
:10381000F55AD44AB77A966A711A500A333A122A7C
:10382000FDDBDCCBBFFB9EEB799B588B3BBB1AAB24
:10383000A66C877CE44CC55C222C033C600C411CCC
:10384000AEED8FFDECCDCDDD2AAD0BBD688D499D74
:10385000977EB66ED55EF44E133E322E511E700E1C
:103860009FFFBEEFDDDFFCCF1BBF3AAF599F788FC4
:103870008891A981CAB1EBA10CD12DC14EF16FE1A4
:103880008010A100C230E3200450254046706760DC
:10389000B9839893FBA3DAB33DC31CD37FE35EF3F4
:1038A000B1029012F322D23235421452776256722C
:1038B000EAB5CBA5A89589856EF54FE52CD50DC544
:1038C000E234C324A014810466744764245405447C
:1038D000DBA7FAB79987B8975FE77EF71DC73CD794
:1038E000D326F2369106B0165766767615463456CC
:1038F0004CD96DC90EF92FE9C899E9898AB9ABA9E4
:103900004458654806782768C018E1088238A3281B
:103910007DCB5CDB3FEB1EFBF98BD89BBBAB9ABB33
:10392000754A545A376A167AF10AD01AB32A923A6B
:103930002EFD0FED6CDD4DCDAABD8BADE89DC98D83
:10394000267C076C645C454CA23C832CE01CC10CBB
:103950001FEF3EFF5DCF7CDF9BAFBABFD98FF89FD3
:10396000176E367E554E745E932EB23ED10EF01E0B
:10397000005EBCE2613FDD83C29C7E20A3FD1F414F
:103980009DC3217FFCA2401E5F01E3BD3E6082DC3F
:10399000237D9FC1421CFEA0E1BF5D0380DE3C622F
:1039A000BEE0025CDF81633D7C22C09E1D43A1FF1F
:1039B0004618FAA427799BC584DA3866E5BB59070F
:1039C000DB856739BAE406581947A5FB7826C49AFF
:1039D000653BD987045AB8E6A7F91B45C6987A24EF
:1039E000F8A6441A99C7257B3A6486D85B05E7B9DF
:1039F0008CD2306EEDB3510F4E10F2AC2F7193CDCF
:103A0000114FADF3702ECC92D38D6F31B2EC0E50BE
:103A1000AFF1134DCE90722C6D33D18F0C52B0EEAE
:103A2000326C8ED0530DEFB1F0AE4C1291CF2D739E
:103A3000CA947628ABF517490856B4EA6937D58B8E
:103A40005709EBB536688AD495CB2977F4AA48167E
:103A5000E9B7550B88D6346A2B7597C94A14F6A86E
:103A6000742AC896154BA9F7B6E80A54D7896B355E
:103A7000EB3C904D53444F53352E30000202010071
:103A80000110000004F80C0001000100000000001B
:103A900000000000000029EFBEADDE41544F4C2075
:103AA000465072696E744641543132202020000025
:103AB00000000000001000000020000000300000A6
:103AC0000040000000500000006000000070000096
:103AD000008000000090000000A0000000B0000086
:103AE00000C0000000D0000000E0000000F0000076
:103AF00000000100008001000000020000800200C0
:103B000000000300008003000000040000800400A7
:103B1000000005000080050000000600008006008F
:103B20000000070000800700FF0F0000FF1F0000DB
:103B3000FF2F0000FF3F0000FF4F0000FF5F00006D
:103B4000FF6F0000FF7F0000FF8F0000FF9F00005D
:103B5000FFAF0000FFBF0000FFCF0000FFDF00004D
:103B6000FFEF0000FFFF0000FF7F0100FFFF0100EB
:103B7000FF7F0200FFFF0200FF7F0300FFFF030043
:103B8000FF7F0400FFFF0400FF7F0500FFFF05002B
:103B9000FF7F0600FFFF0600FF7F0700FFFF070013
:103BA000120110010000004051C203130001042063
:103BB00048010902200001010080320904000002CE
:103BC0000806506207058202400000070502024015
:103BD000000000040309041C03410054004F004C82
:103BE00000200020002000200020002000200020D5
:103BF000002000280346005000720069006E007427
:103C000000200046006C0061007300680020002066
:103C100000200020002000200020001A0346006938
:103C20000072006D007700610072006500300030A6
:103C300000300030000E034D0065006D006F007213
:103C4000007900008721000000000000A7030000A9
:103C50000000000000000000000000000000000064
:103C60000000000000000000000000000000000054
:103C70000000000000000000000000000000000044
:103C800000000000A43C0000000000102C01000017
:103C900080330000CC3C00002C0100103C9C000054
:103CA000E8020000BD41544F4C20465072696E74CA
:103CB00028054AD4284B3D0276102C0E270780C3D6
:103CC000C9010087930304456CDC0200B1670E98BC
:103CD000D83EB112C61F623E4752069D7012C5A85B
:103CE00090700647AE10132C962B84B8AD65007407
:103CF00081D1505DE4CDA299E19057EFCC146AD701
:103D0000671C9B4876A8FDF07643260E23BB241142
:103D10006C32B5E75369A9DD057F415B367C705C89
:103D2000F4C7B99A9284B6429FBEB25BE3C8101240
:103D3000275814B5D8484DC342DF5DBBB4F9657C44
:103D40005B5272F3E50C047C9B6994E554A20A6112
:103D5000B17D60733DAC9033CD7E308744D96731FF
:103D60003AFA6A4FE9041FAF410F872C61CE7E2CCF
:103D7000ADF55B028FAB6EFBD451E860A18DC5C879
:103D8000609D5332CF2356F2F396DB54AF708A2DE9
:103D9000FC34C3F822DCF8430C8AE2CB7B252B00F1
:103DA00055B0CC52C280A74E78551226AB660C3166
:103DB0003A4A951DF5B60DD4DAB523C2B8A66A7C89
:103DC00010E12D90D9740A5BBEBFDD35098377DE23
:103DD000EB44CEFB4284015FE6072112D10E356130
:103DE000E5BD6FDCDA386AAC0409563FA66E41794E
:103DF0000382F562D91ADE7E72795D05C81D4CAC6E
:103E0000B5E3A86310DF7A085BA937C3D28FE95501
:103E1000B677F6F5971D5FCF557D4AF5D10009C9F4
:103E2000C549387A1978515B05474E2DDDAE3BED1B
:103E300089A00439E614DD4F5C7247D8AD374EF6E1
:103E40005CC8F3DC041A674B3A702005050F9CC769
:103E5000A80092E49F7E12FFC88E4145FFEC2361CB
:103E60004750D3FE0965E8424DAC8653FE972F10AC
:103E7000D5233DB11BB162728D7BABEF37A424E13A
:103E8000F4CD30CA899648EB736CA23F33842C5A28
:103E90008AF0B07124D000EC65CDEB6FBAB4C54F99
:103EA0008B6D921E1C1A6905F4CD70594792B9BCEE
:103EB000D11A1605EBE55A94F5B7AF406D94762903
:103EC0000FFC6C17EF524FD87FB4A13CE9BDB9F697
:103ED000884D3E2F276BF2A490E484642E0C11DAF7
:103EE000A4BF5DAFA96B38643DFB7B0786D5E1C4F9
:103EF000E5CF48611D613655666682508EC996953C
:103F0000D1A8DD93E697B4DD0A8F88E1AFAB3544E5
:103F1000737A3623DE3C86BCC08FB154B501A2FA59
:103F2000007D290C091A896CF093C194A4EBA3308D
:103F3000F87B73D5ACA6C289788E5C7BEE1C10F53D
:103F4000717B2AD07896610CB41EA6A9ED7001EDA4
:103F5000389F315E9C4D30943FAFD15448576D52DD
:103F6000EF9EE71712EC9BADEE4AE747B0D48228EC
:103F70001BBCD23A7EB33A790D4F0A2D229E0C3FDC
:103F8000D0DD0DC8A690DB69FB94F34E0F188300BB
:103F9000B0ADB53941B4B46267FE9620D6F1653054
:103FA000DD0F3EDBE3E3B2F03A98971EBB833CE5BE
:103FB0001521F5BAF70BD0084D60520350F8136283
:103FC000351C32E95902A9228A856928B8BD661CC8
:103FD000E08308732F917F75E7BD9240252A8649BB
:103FE000E53F7C227FF2D01863CDA4E020CB95037F
:103FF00007C99AFCDCCAB8B427BAEB6BD8A97DB262
:10400000AFD1A81A92870ED7B161D9227CB7900997
:104010005FD4DE2670B4E61360B9BD51AAB057482C
:1040200032FEAB023E286F16281B4881925A7B6DE8
:10403000677E9176EA783AEA1C957577DCFE01B5E1
:1040400087CE244A16EF8C96EDC63CFED4E9F7AF36
:104050004EE8F6B4829F6F0C580FE1B504E40237C6
:10406000B1686BC7823E380C4998F7023151E47F42
:10407000255FC7DE73F2DB46B2C5D3534711DF427B
:1040800017918B4DBDF40E35CB3DF78F9AFB08BDD4
:10409000870209CBDD96B15A3B3A3DC56294024294
:1040A000338C6F22B72DCE163B5E1E9F8174353C3C
:1040B000D2A0E3D9DD8D26D693E1D9F5EFC57F1BDC
:1040C00086381F93B4A93E6EB67F38B3F299187C38
:1040D00059D14CC5C964702707B12D8F63009EE884
:1040E000C27F80E898016E11B58D82AC1F90144D8F
:1040F0000EA7E47F47FCB68D1582E73CB91E9701F9
:10410000C8188C66FF63742B6425BD80931B2278CE
:1041100007377CD3A9B2BA948BD274297D28F94B86
:10412000F84767EF75D064CDF7A6562DC759907A3A
:1041300074EE4251B169FDCDBFEFF3999ADF566439
:10414000B12C82F998929C9B3261D7D0A700C752BC
:10415000AD9364D6632C82643B945672AF6ECF4DA0
:10416000FDC788FB4342B92CDDFC4A72801DD74B4A
:1041700031026905AE2D75782DF4CD9242760DF998
:1041800081AA74E791BC70D06F0AEC2E8A7DE8CBCF
:10419000574E1E675A351DFD4B02E8D079DAE018FC
:1041A00032D16726C888A1D9DDCE534ADB75F359D1
:1041B00045B33B4B6D57F8516F2CFD520D21B0C3E9
:1041C0007824E3745F59B4409C7804FE20C566E10E
:1041D000C6F4F9AC8A1AB8261D49359AE3FBDE47C6
:1041E00035CCE4E1A98D400A8E356C1E1FBA5F798B
:1041F000941944E35CD95F5F04DE18FB7DE1366D02
:1042000010C93915A61AAE1551107E0F911858A372
:1042100003D813574951A484253D6AE9D9BEAE9409
:10422000C77692216A97C3A281B2505E6C81C69410
:104230006D75A36279A2395C15DF3E44D95C558F58
:10424000BFFE4447102BC9C420C73FC5D4237A53AF
:104250007BAB743E56CECE045EA1FDBD71EC02D4A4
:10426000C078C5C19B9A10A2529DA2A840E2DC343E
:10427000FCBE257929C7FBD3A069B6E88E4F00861E
:10428000624C50AE5F6173C6F297037126B8176730
:10429000681C6006ADF4A6BB01DFF2C38275632E15
:1042A0006C099512416BAAFFB45A30E963CE79AD1F
:1042B000C6CC11E7DF0BBD81DF5C74B7C484AE10E0
:1042C000BC8E691C7937767E550A2CA8434829E3B1
:1042D000973E2E6384B0997DA1E94EF47252520E3E
:1042E0009B5909330CD1633A33B9043AF02F50F398
:1042F00021C7797544DBF4056B1E5D1447CF08F8C0
:1043000009F5991A2024C81A8FB99EDBD4F8754E86
:1043100084123618D1D2607179EBD8139BA12FEF9C
:1043200018433C5C1322BE9E85CB773EB1B79029E3
:1043300043656731B291A41F36D6AE4BADB2E31FD1
:10434000A4A53EAA8FB3F83608FAB98E57E3A22780
:10435000869FF2B8EA4EA7F674D40ED2B3045D6815
:1043600078374FFB1CF10BC27309F6AF08C54D56E9
:10437000095BA5F5B663FA0518D529F8DF3DD8A184
:10438000D4E889BD93D9F7B8ACA4304CA8ED472147
:1043900043B42791CC8D397F5271F363C827834D85
:1043A00063C9904B0254095ACFC887CAB4D8E819D8
:1043B000B1EF4ACE8313E5F378EE3136E732E70DFD
:1043C0004D4357120A4D8C862287503F9CCAC937ED
:1043D0004B1D682F3749DDF1AFF1B35998BD41B797
:1043E0002626D1B6B867575951C891A6F3FE9E53F9
:1043F0005932C5B3A147E7C9E044166BC52FCD08B4
:104400008261CE24B2CE1D96DEDA78AB62170EFF43
:104410001694D3692D63BC28ACEED98064BDEFCA75
:104420005F911E755AB89697CC6DBE341901DAFFAC
:10443000DDC8BE8242F6D7046642844344B1FF53CE
:104440003472CFEE0FDF3763D79269356304996614
:10445000474327256DCD2E747AA4B7F1C95A428EF1
:10446000B6E7846C322690797C41FAE53F1A8D9B41
:10447000967DF27691E6D766F038C2632199E6CA56
:104480001A80EF81E1AA1DE3C9EE78F20602A3BC0F
:10449000E56CE3AAE7143B8883CDA91F59915843E3
:1044A00086777D02DE79533EA9AB93CE7EDA0D2965
:1044B0000C1B400A4EE7F247FBB6EDB8453EDCE880
:1044C0001DDFF199420111D1B8FED9BC1E3C053166
:1044D000BBF8861C90E1BA0B5FA8E2D231C7BE914F
:1044E00093D0DAE31E8172DFF02B54D1D734038CE2
:1044F00093C8E64BE63736B044753568C13EE1E215
:10450000EB6F9DB8862DF16903A0DF24EFF78625B8
:104510002DDF63A47605374373BF348254734A7723
:104520003E2DAD9EFBC4CA7743D192F47D6FE03639
:10453000A3CF51BBA81AF7A290671C0192D36EC0FB
:10454000918D80FE7F46D1C827C8A2775A7FFD464D
:1045500059E984B9FB39E2B063BEEE57B6DEFFB766
:10456000EA66C8AFCC128CF925C4E7E28F1EB456B8
:10457000D6D1253F91B78B8649D8C23015ADC0ED55
:10458000498C2CC970D973DA0E512976B954AB48CD
:10459000E065D8F0E373B1159B1E318F498A6596AB
:1045A00066439C2C8BBFCFD63F2B8937CC2C5CBE6F
:1045B000FC8C63D1DEAF4E264EBF333EE37C7BC620
:1045C0006751398AC2F2EB5168B5600B283ECEA61E
:1045D0007CE8929185B45A411DBDC15224D4BD25B9
:1045E0009D77CE5E1D3897DDBF40B1A5D608E07936
:1045F0002B4B0B00D667A2A043069C21D3CFEB7CAC
:104600004BF45C421900F7F1ABE07F407DDBDAD17F
:10461000EA0CED440DA811371205031F39BE0E5BDD
:1046200067BB15A6A832D3C2656B77DB7C594BFDFF
:10463000E31E7E92F1E30AF9351EFD32F3B8C2495A
:1046400015FD946DB5EC4C4D4E997108C3FC05BE3B
:104650000382BCABC628C9811595A863FA0FE52C67
:10466000045DE3B7167BA987BE23E05044A5E1A70C
:10467000ECAD045E04B0BE00D746BABF65EFE4AB54
:10468000DDB1DDA4F6BC86A9A8759BA0300FA0F90A
:1046900096D6170246A2DB0A1D73A4F24F0C3CD932
:1046A000497623A29EA11BF9DBDAC7266E00C4E877
:1046B00031D153F7AC8EFFB9577BE0A5972A7F190C
:1046C000D9A012ACA8BAE450D13345525CB16A5AB1
:1046D0007FBA23891C15B6A0C7BEC06BB75A0D2B75
:1046E00068084D8C5D942532C414042C6D8D539B49
:1046F00053E39FDA91DC7B3C8944D2363B769F21A1
:10470000E4FE3ACE57760269EBFFE2EABDDD3DE614
:10471000507F72379B2B1386B76AD7BFFF665293C1
:104720000C51AED9907BE852A30A31DACC14A5958E
:10473000CCF588FB02763B1253DF778D64B861CBF2
:10474000CD9FE05BEBB5F85C42050ABB10B611DD0E
:1047500059ECDC4AB4CDC0B0F56C5AE38723532E34
:1047600088695DF24E5C8B3FA8CB25497AB04CDC62
:104770000EE95619E937123C02113CC3942FE87434
:10478000501F4018CBB84D6E9B162B53977CA91B1E
:10479000B8355C95783A84C5B91AEF648544E698D3
:1047A0000CD764B112162DA56046AA7EB4B38EB4A0
:1047B000A89D452EE2A78814FEDD034DF049B0D137
:1047C000AE3461CA2FC68D7CD69A9272F91BD5A7DA
:1047D0004E32BEC8BB66CE3056E9332FC55D24BB12
:1047E000DE939BFD689463B61338D4E29985BCFDD3
:1047F0002F4AA6EDEBD10A6738EC6A2DDB86AACCEE
:10480000D1EEF8AE539A43CBD14C60766F757FA052
:10481000E9D0F020EEF6A80CADE416BF7C8ACD8B73
:10482000FD25BD2B7CDA2AD92BB8EB6F840147819B
:10483000D9F606249C7F4D1C4E18FE790C163DE0DF
:104840009E45BF2B38FB89DC4247B35514F37FFDEF
:10485000320AF8DD7E797D024E5CB3AECC85DD7B1D
:1048600094DF1431674E5014D645AFC825550C4718
:104870005280DC9A818FB677CC19FB60AD9603F439
:10488000D559A42000EEA5C93698AB509F0EE2473B
:1048900075CF718635AF8E3C00D5707E13412E5595
:1048A000DFDB968463AA86469BD1E88F8B7A64E52A
:1048B0009C10688CA6FB5A8F614ADDD003ABA1DB4C
:1048C00079B60994BFEFDF7BB1C3DB6D875033ABA3
:1048D000E75A5A315E250885212EF1EFC886432517
:1048E000254C1ED4DAEDC6BD913440692806C88730
:1048F000D09CDAEEC534386F564954680131060A47
:10490000F29CB7F5E628E264A75049F06B5C0423FB
:10491000E721DA816E1456D169DC190B15C4B7DEB4
:10492000D43116ECA1A1F9D56377D914364ADBCA84
:104930000D3CD9090A9CFB915C9177A2923C8F981F
:104940001A7A6210C3E307E283BE6E12C1F465AD4A
:10495000CC55E3BD10DB9EC0471CB132161BD1E61F
:10496000C458EB91D9DCCEADFC47DC71D92CFEAB41
:10497000D42222D88DC714DCE9EA11E7021B7E108D
:104980008C377D2C653C779E692A160CC52730AE86
:104990001B20200DDA3D8DA9545D7FDB9875FCA8A6
:1049A0005B06492F61C63AED2F581199780154479B
:1049B00005D0D173E449575BBB799434E55C490E6B
:1049C00007CE1FCFB200E91A7C9E1CEFFF688F084C
:1049D0006537301143A6DB4179D6052F1EA3825FD0
:1049E0006D6FEEB89F0208DF9073BDC12FD5CC1755
:1049F00083F0805A78521665D81DE4A74A1C6FF6DA
:104A0000CE0E63B084D0ABFD5960E80A6A6E9007A1
:104A10008335A03C4EA8455941EEC70B324295DB89
:104A20003158359C042AFC4984D578F2D107A50079
:104A300035B19AAD7884FECD423D18081486E46104
:104A4000C2752EAA9AC0A1C7F2471C28AF3581357E
:104A5000B9E6D2C5FD622D59F78552F4C1ADFF818B
:104A60001B2628EF65B0062BFF82381959177C7278
:104A7000E89791725D7C24D09A97EE51A3495246F3
:104A80001F69B014E5E9FB59F6E01AE44E5EFB1B22
:104A90008B3F0604A5ACFF26914BFDE0F288FE3863
:104AA000CD32C7C76E45C3EC7E87FCBD1C2B43844B
:104AB000BB38C152EA4A73B8175D26C4E9C24FED4C
:104AC000E98FE7EB8769BCA7F9440EB9AF675CE9EA
:104AD000FFCE79447F5366BB20B1013E21E7D96602
:104AE00097BBD59A4871B45507FDA5A5DA72D69340
:104AF000F660524B4C4D5B508A996F53B2A963A23A
:104B000056F9C9D473F912B3B3FE6A7373BC5298E1
:104B100058D74730628AB24F4A1D20B21BD9AEB176
:104B20004262FB4E98E11E0608B3B591498CC7134B
:104B3000158BFEBD68275C86831A50FA2CF4C42BB3
:104B4000D6441BC1F137A7500BE90ADEDEAE8EE971
:104B5000F427889421E0A1B90DCCC31E8F2E0FCF6E
:104B60007E1158ED068D0365DC9A1A0810A2B495E3
:104B7000D7FE231968334D2B62848360E002308AAC
:104B8000E2D8BCB3DCCB4557939031F12689986BC2
:104B9000F70E2B1017114F78C55BF6D4606EFC80B2
:104BA000AB08D50891742DD73D2A143B7BC14D42EB
:104BB000C68E43173324796BB401B4932BB9812784
:104BC000A94A3E1EFC0975797F8E480449814EDB57
:104BD0008293CFD5FC424CEEEA050894D6C11AE583
:104BE000F0F3CFA234C9E8D5703F697B18DC1FE62B
:104BF00031429B0DA098079B7E85EE9F738BFDC76E
:104C0000AAD1054FA96AD742D0ED1B493F3E5B0CA4
:104C100081B88A9295D46C88FBD4DDD93755D98A6E
:104C20000A4FB7BF4D4623E5B8C8C9ABD0063136E9
:104C3000F05F16D3B3000E2CC854E1A60D3009FF67
:104C400099A5FCEFAA1D58431E8ECCF8E669A499DD
:104C5000DBEA0C42CF29AC1FCF8F4A88A8616AF4E7
:104C600047758F3319A464103489BE9D00909966EE
:104C700043DDCA8BC8955DDF90247E31C47F3791B8
:104C80004AA0D667E307F68C6ADEE38E1B25DD8A31
:104C9000CCD7685FD79A92A8BFDDDBF4C195A79403
:104CA00049264CD6CC52E611DF384FC7314F8187A9
:104CB0009D27285123ABAC4343A821C2CB4A3AC716
:104CC000121FF9757DADD796A102F79F580B97AFCC
:104CD000919E65E46650D3727DCDDE0FCE704BBAE7
:104CE0004A4946950AD4FC1F9ADE2D77CAE38A7694
:104CF00052BD55546A08D44BC360458CA5ED2BF1C9
:104D0000CEE7A1CEF809F23514893615A65C16FB5C
:104D100000BD1BC51F9F4D5399F0BAC021929FCF74
:104D20007031822174A353CADB56677BE370497EDE
:104D30008F0A0F57BB22121C71CBA485406E8C3892
:104D40007BC65ADB87975BFF16C543DF8C389CFA1E
:104D5000043D4784ED1B3CE7154A694B331C0C624C
:104D6000F3D83CA41149FBF20E6702D3868F64BAD4
:104D7000C27BA962B4920090DC54E415D578B77A6E
:104D8000408ACB2625A73CB06711D97A45061BD9A6
:104D9000AB1F8BD57E32C450BF8DBA9FE081DBDC68
:104DA000115C70B3800187FB1E7533EA3095683F54
:104DB00023AD23DDC94CA7ABFCB7C7916A0F77C5FC
:104DC000676DA59134A48723A87F0E7261080280C5
:104DD0001B8BBFC6B66C0DAA417E9A6B674EE9432A
:104DE000F9723ED28D4E7603757FD325FA2E248834
:104DF0002135FBC9A27E2F183FB3DE977B2CB1C9AA
:104E0000D7476397F92F2D4F3428507F450808E482
:104E1000622BA7E64BC79118C62B99328F68DEE24A
:104E2000C585BF5A559FB0C5A331168F8B99B3CC9A
:104E3000D5DDDB755BD69363819259D288CFDA1CBE
:104E40003238668BCC4D852C35606C6DA8A9364404
:104E50006C577C2C7BB9D28CE9547E0F7F2445970C
:104E600088C653D97174216020DCA7E822F7DB4A99
:104E70003D1564D8CAD46DF76073A6E44A03C1280F
:104E80002FD64315FB9E48BDCD3ECF6C09B061F2D5
:104E90006132D53270967BA55AC31D9241815189EA
:104EA0002B9DA936FA36029F141F305A948AE87C4B
:104EB0001C98A30AF3289CDCC14F6319F60FB02499
:104EC000CC93DD095779F95EA7AB2A1B550E054A2D
:104ED00069198101EE6E279653316AABC951D346E9
:104EE000902BD4CAEC63B50D7C7014F4F5F9836E85
:104EF000DDC171E86C580B1FE3BB9600E0FBAC2BE7
:104F00005F6D81C4240A131D0A906CE145797F818D
:104F1000ABC97236786C265E291F11CF41D0522959
:104F2000A6CCCDD120BCC467534E096E9F9E3F8155
:104F3000584841242F1B70EB3D20E6C0082607F699
:104F4000C3F35BAD38683C4A21FFB005F34E664CB5
:104F50001C45265A15F1061C241B0FAF1E8511E9AE
:104F6000FC0F426E69C7AF1E78BA6A59648BEC5564
:104F7000972E5996339A41FB046F6CC4E4D95B06B3
:104F80009801047C9FB7D84ABEB51D51C65CB07469
:104F900062CCFA15E09472D796DF072D4D5953B0C5
:104FA000A23CCEC6FB9C214AC70803946DA721F6FC
:104FB0002B0CF44DE17F00CB3B085DE5703C354F99
:104FC00063C421381D88EEC99DDC501E6F1FE87038
:104FD000521B3DFAF606B94C77A71B8E8149F209A0
:104FE000A0F99A8B54AF43A5C082AEC0868A2341F4
:104FF0009AC45DD818DED88A3A61DFF784A988C5DB
:1050000038E8DDCA0EB65060960E23E749B53A86F9
:10501000F290447753E35084DD4D2754282E92526A
:105020007004A34E67E12315D484C75847D704FD05
:105030006A8C4846520EF0DD28B9025E55CF171B28
:105040006A60BEFAA72DF874644C6D4EB0602BAB4D
:10505000D9671BD3F27B700F592E359670B641A2DB
:10506000D96F4CA3340AB113BFA3FC9C7162F288C0
:105070004F14FDCA3CEE9EFD6D9BF3DAF783AD8DB8
:10508000FB5DDBD3051CCE587656A095D18948919F
:105090005A4371ED476DDF63629D3405D6E89798FA
:1050A0008847E6853612EBF0F98B83C08A70EBE215
:1050B0002930E0DD2B2C441FF4AFA9D0561074C565
:1050C000F7B86B208E807427F48FE1051DE9F76037
:1050D000DFA7ADB51241A65BA880D6A2D03295D489
:1050E000E333831B66A9DD58260F051A7FFF54079B
:1050F0001AD4B64ECFF35E7B80181AE99B13C4E92D
:10510000F6DD2E4EEDEECFCFA19C73BD361229DC1D
:105110006B0272BF7DB2D4D692DB08AAB3243804E6
:105120009ACEC372338C2D676AD4EA7018086DA3C7
:105130002B96B91C66B4578EDA4A70999A5443225A
:10514000C31967C9B38106EFE768BC861B0C0295DB
:105150007C8617BBCF21E9E0E65D2615A65C1389A6
:10516000470A6A60EB6EB2A46ECB659D9DD7E3499A
:1051700013C523B0C739E30C046DD3721D31A930B8
:10518000FAA4B1BD8F4AA4FDCF347258E55009305E
:105190003384093176D3C4D3DA4A4CB722598F66A7
:1051A000D98E375772F76971EAF30820E7AD1BB261
:1051B00079E113566D9A2FECABC30B2A3C7865B19D
:1051C000A8E999512464D3DE990085AF29D87DECF4
:1051D000FDE4BD04A56F14FF09EBAA2AF5FD82FDCD
:1051E000C3A17218C5397A1D65F42B5F2E59DB2BCC
:1051F00021FFDE1C7400569AE1B0B23661FA3781A5
:10520000AC6F9FE08D2F91B225EE1A536AD7ADE2B5
:10521000CCFFC97A7F5BDC2076EC7BE793FC974A76
:10522000255593D5F89744D06B9F0152B574AC6C5B
:1052300032A6CE604CF882C9E0265C2394BA05FF02
:10524000737810D8A304F35B009C6A0A929D5740C0
:10525000CE0DF7541DD3E7500C5C48ED55D98FE5C2
:10526000D9320F4BFF722E2801F8A46EEE63316322
:105270001E8190A2F1F38388F26964BC3FF000D3F1
:10528000650EA2596D8D26E04BD27EDA9701ECE3D4
:105290001FBF3FCF6BDAD26928656FF97212388D64
:1052A0004EC2C6FD45FB97369B8F275FA72BDD0CB3
:1052B000ABA3E4919BDD51010BF1A73E2F29C92E31
:1052C0000C13160611062BDF5E4650CF54099501CC
:1052D000705516A7AAE1C6CC087380A7FD0FC110B0
:1052E000C165AA9F98B8B5FA299DE246E0D5ABA45E
:1052F0005810458663A1BFF48E7C842B05AD15BD87
:105300005BC8BA14C1D36EEE1A0DE643D57650A22F
:105310003B878C91B6DE5081719ABE1C6F42258FFF
:10532000BB3C57837F6C4ADD726545F29F0E2BC0F4
:10533000E02587EBEE7DF0948B29D0AC00F07F81E7
:10534000481FBC420F77A4F03FC0C3C0A79BF1C069
:105350006942155A4EF0AA689D94DE5A699C46220D
:1053600004566B1AE87476112A7950873D9DB2FF76
:10537000DC7F9CDD8D8EA3C6DF087A69B4D9133F2C
:105380004A499E300930AAE2B1596FFA4D47127E60
:105390001332B378F3CAA667A69ABAC0DACD972AB1
:1053A000C192EC61FF2E1883649B865CC83A5FF65D
:1053B0006F4CF392998B28FCE189F659CFB9EB1128
:1053C0007A554D3BCC15F2E2B858EF8F1F3FB71717
:1053D000CDC210CFA65E7641C8BBA5D88314888401
:1053E0001038DDF9E78973D51F627D085B59F3DD5D
:1053F0000A9223F3C05C35E737204A18BF03B4BADA
:105400000C9FB434A26AC2AFDB8EF9640ED79ED271
:105410009DF0AECFC79F0815E0C82A41DD7E4C9FA6
:105420002E7487E9095A18991A45FC6FF3F5D00BC9
:1054300063F778CC37C4C5B70132F45BDD8B7E0FE0
:10544000730625B3193C0FD689CEDCE4CAFD980A51
:10545000414A678AD316BF972D7298148A4B16DC7F
:1054600018C5E08056B15F5B955CF4F5A306F1D7F3
:1054700096DE8C79ECE56689EC9F54D0F07F36039C
:10548000DCE91C752E48248652EFC73FD75121EE28
:10549000E139B2EE608291C6E68377A6386D1DC110
:1054A000EC4C4CBE94DB143AF33A59A2EEB9905846
:1054B0006F6DF06EDB911571DB3622EC6DA2B6FDDF
:1054C0004F7C59CE8665E48945AC9E8E7EA4F394CC
:1054D0006F9FA6946FBB9336041875BF3192DB4360
:1054E000354EA099CD985A42B40BB2B423B66FCDC5
:1054F0006310DA0E98B796813D4CB099FD793FEA7A
:10550000D9A70370410BB601B8CD844F9E480C6BF0
:105510009A6183935C0E357B5017191E3608AD2AAD
:105520001DCBDD3FCAA8B19CFEE8A9275D5843A664
:10553000C4FF88154436CD1B5C101DE875DB228244
:10554000A13767E2FBD3DD08F1AE0748575EFA6684
:10555000D7A0E514285996BB518926D2FC75DC26C4
:105560002DE24D7C8AB21B5D012068EA243AEBCC27
:10557000EA59D40C77FC146A4294B33C01ADA64DB1
:1055800091F6A9EABAD37E682CA1E93994C1E7362D
:105590008AC89D51F12AE8C632454763E0B9ABF5A8
:1055A0008A0D2FCF63CE1D2A9EEABA248764322D3E
:1055B000952513046903A6A989C47EA4688CA3B7A2
:1055C0007B9111ED3258B8725056C806914A3EE5AB
:1055D000640E3920C1284C196A57F18BDBD7D030C3
:1055E000BE129C42046E1F091CB2B7E025536A0626
:1055F000030203F1E39EA70FF7DE53A390A37F58A6
:10560000E30E58DA0663F786621ACA799FC36423E9
:10561000637D85C896BA5B223FC2641EB4AC6597B1
:10562000333DF61ACF909DEABC6A0CBD6C5C4B67AB
:1056300026EA47B3B68D90CDBDC6207E308D449D01
:10564000772AE1A9BE4120D1BB178E2578B807A8DB
:10565000E78F7D43EFA019D4AB0BF97999D2A2B2B1
:10566000C53A04B4B379B8437429482D511292E570
:10567000B979AF4B3ABBB522B93D3C049B0E502BD8
:105680000CFD2B5EDD97389B030D52AC0D947666B6
:10569000A92ED9363D299CFF5736625131CBEC52A9
:1056A000DBE2F0D6A85CC37300C5BC9C3C37E7893D
:1056B0002A22221F6EA1ABFD380F2F7798A9404AEE
:1056C000D6D9CA5270B85AC3FF2C62CC4CF1DA9BBF
:1056D000F8841C68E6027ED7501EFC636846CD2124
:1056E00080DD44764B472B30AA77BAD83268F01267
:1056F000FBE4BDE717A0B9790F3F3D896E060D3376
:1057000034F595859EC3FE9D5700DB362EEEDFD81F
:10571000FD38B81DD2A6092F8FE23C21A872E6DA27
:105720008C444229A401C00B06C2DFFD769BE9D759
:1057300069A899DE07678CB723531F2F3B548A0152
:1057400073FDC7A96C2B5C6ACF449D3988F0191F83
:105750008CBDB5454ECF6515E60E173DB429A91F82
:10576000EC8A1AF51224C5BD1E5962DDA8A4EBDE31
:10577000C2D29E70A4C5A0768BC0DC646BC17B9046
:10578000A025E3F06EDF693D305761A1AF10CB1A61
:1057900079912D4D7E3079194935752ED14E6D6434
:1057A0006D2F2127FA3F59F1C2395676942772A7F7
:1057B000F4D383F79DE363D615B65B636E29E2D01D
:1057C000536E95683F8FBD2D98841A873484CCD052
:1057D0004C1A1B58547B8F13DF4AB4E458EC1E3725
:1057E000DA93797E194119494FB35CFADC3B9F7912
:1057F000B96EB8396150E460714CF2BD7E20B3E5FA
:105800007C6B848DE8BBAB5C43E7DA4626E0A937C6
:10581000A1202132C65DE7A3424547446E349E462F
:105820008AB183FE5360E420C0878D3DF6FC3D02C3
:10583000B90FEF57E4BE70023B74F6DA1B9B2EB92A
:10584000C4FCFAAD04D3DD13277F2346B39A81A3AA
:1058500045930957C9805E424AE4BC793139110148
:10586000842E0BAE8DC44DB9BE8CBA6CAF74BDC85E
:10587000C7ED7406C77A5ED41F7F04E5D4ABCCB7FE
:1058800063FDF3B31364B558901FD9E4CA4E1934BD
:10589000F93CFD7A94657813585EDAB25A39D11E14
:1058A000F1E29F2E2603B0B255F3AA15DA326480D6
:1058B0001BDEAE730BC765A336D1D3C0B62EFAC6B6
:1058C000D624747C2F7F9F0103100A20496B5793C5
:1058D00081787B95086179758F33A9FACCB568B565
:1058E000892D063C0E6F527793C9C2F3F714E2D6A6
:1058F00045EFEA5D33DD0F9424009A4FFF1985FAD6
:105900005C9D0F1BD560049684CABD92CC51D29B7E
:1059100009CC1E17E012D746BA00259337C32E8054
:10592000CC0DECD4ECB2DE3A0228861FE0AA09F3D3
:10593000A74BF5048C0EE12ED31F9D6375575FC0F6
:105940003C83106396D08038AC97C4277BB0866BBD
:10595000F6C8084EC7CBACEF4292C54723F9BC90BE
:10596000DAC53FCFA3E3880EADAD498A3A06466853
:10597000D6C8736EED067F4B1FDE9772DA5D376611
:105980003FDE078FDE12F374D2D2AE60F4D55F0D26
:10599000EFE986E60F333B3215236EE6F55CDBC19B
:1059A000A309E62EF53996C48B1F98D6EF206854CC
:1059B000862111A15233A2ABB8E0AB991A500A92DA
:1059C0000622428C8E8B86F87883F345292613A510
:1059D000580E047B16B48A8615C160BDD83CA05C05
:1059E00072A3769D47C456E9B768AD3A52AF57B532
:1059F000BD9BAE36EFEB89EB7A406D2F6C7FB55BCC
:105A00007FE0A3DE3AA3A1D98E324B08BB2B46AE72
:105A10009C13AE8EDFBA64C9E49B015EB70AB5E899
:105A2000A0C821BD3E9000F6490EEF13F94E47D1B4
:105A3000DBBD9F0ADCF80924C672D380F845CDE8A7
:105A4000CDBB7DA477853989189B72CDCB38E5789D
:105A50002E8502501BADFF6DF9BE94F29779596AFD
:105A6000CAEFE58F82B1A9882E9267553E253F6126
:105A70003699E214F8CB36CC3EF4895A74F35F754C
:105A80000BEA4518451F87CE40AF04F68BEC8D21FD
:105A900080107BE61C46C4A2A091FF499587F37C49
:105AA000391E3F7979931E3306AC0C8B88C43DEDCB
:105AB000065B60AFCECE7ED45B04EC99A5885473B0
:105AC000AF3C7AE4A2902F86A3BED23F527E63CF32
:105AD000C22FF5EDF86460AEB806EA29AC7DDF2888
:105AE000BD2366E714AA824BD7D3CDBF0EC7193D9D
:105AF000D37425C7C472BE5D0853B61FEB6A9D19E7
:105B00001AD90954CCE414F143521C382D184D20F5
:105B10004181978C07857FA1591B164AFF83629BA1
:105B2000EEEA4B7B25688BC4F4A2DD050848E3FC54
:105B30006406B11F6ECFE90125CD6D088C54C501F7
:105B4000E99F6DE94FC1F1A4973FF85611E38FA18A
:105B50008253DC7EC90889EE54A0CD5938992A2A8F
:105B60005C4D24213059A512EA6C6DAE58F34E718C
:105B700060EFECE86FFB2EEAD94FCC7F8F8FBDDB57
:105B800011C33A82ED01ACCA81AEB1BCB6D4B6B68F
:105B900028F897E6B0AA1036F185E1E42C628AA7CE
:105BA00028F014C745B0A43BAA4DDECD1673D6E04D
:105BB00014ABD37C0AC61A265B3383610F4803EB10
:105BC000D6EC33B97B0FFBE8BFF85D8887E9F05C62
:105BD0000E6482AE25E028EE8B86CE93BEB9B9C99D
:105BE0008F8843CA9EFE9FB2FB1F5C978327083CA9
:105BF000410DDD7D09F0865DA930D965B8D9CB07A7
:105C0000F58FFC2A808C1FC70FCD6737342376EBC6
:105C100096B3DD681E1CCCAD0C4BC8E5EF2D695169
:105C200058D99452DBE50AF90B96EB90437887E755
:105C3000E8E1019E74E3A03F8E2E9EF0813834048B
:105C4000B81414E58494460F3358EE6A806D036EE1
:105C500077BEDC9FB5EE4BECC363E43085E89BB2C6
:105C60007017479F43E48C7B94A12B58F5E65CDECC
:105C700021326956F4C8287E32ADBF599885BFCD10
:105C8000DADC3E4A4D8220193DA5109B8D5F645899
:105C9000F135919A285180C71E13E85BE00BDD12A5
:105CA00039782E306E46A6A4B781AB60A39C376EC0
:105CB000C6F81FF318C7E48B31E74334EA831AB1FF
:105CC000AA583ADD492CA9B855F01EF6DBA9EFAE6B
:105CD00034EE7F27A680D8C0F5F684A829F53C438A
:105CE000EE48BE48FD662A36FF2354420B43D3518B
:105CF00005A4E87CE28481B3BCC894057A5F438A3A
:105D000026131CEEADA6301D31301B075021384B39
:105D10009B169FF841AC45F87FBF0F60B2589FB10A
:105D20002F6C61DE887A29DCFCA134844768176A0D
:105D300066A4AD76A5649C5520B98B25F47EC9BBBD
:105D40007864612711AB12327C876C9382F2D07732
:105D50004B17759CA4F0A6B16237B0667B3A9747A3
:105D600098ED6B92C5EFE23233735C659FE5A25C00
:105D70006A1B0B3543947B5F16FA401AA39AD7AA85
:105D8000D4503BD9CFDDE4F56A39C0F544856CEBDE
:105D90002AD7ED599275D725EE3B7385CD48194426
:105DA000B74195C51207974B07D5DB905DD8F11E1B
:105DB000239E41EE428B2598A8F3BB2E4BC3C4799A
:105DC000828144D345C57C092926586E41576EFB14
:105DD000A923EA4EC043CD5E633B2A244294E95B8B
:105DE00037269AAD76848001AFEE3B00D1E53CD5F5
:105DF000B47A81EB773ABA9E5FEE5AC3B2E3FAAB5C
:105E0000ADEC337765860C3CE858EAF869098C7389
:105E1000F0FFE7AE34A9143B3CAD22B565F8D01BCA
:105E2000CE918FEE0705254551315966E6463385FB
:105E3000009C924E1C955F577D0538CB7D89B2F250
:105E400096A777629466D7A67AE51E023FB2E91458
:105E5000CB236B7CD7940A2F56C518B0F3686FDF3D
:105E6000E8167B5A1CDFEC73DD2F32A4C5E89FCE09
:105E700081218E0B5C6CCCD25E27AF7A614091534E
:105E800053164707A12ADE57E6D149C6B60763B1C4
:105E9000DEF64E781E0A7C856368D050E320DE1063
:105EA000E017E137A0D6653AFB4367113F34CFAB2B
:105EB00030BCB37D049F1845446478AD0039BE9072
:105EC0005DD344F1B3463C9383237182BFAE722508
:105ED0006C2C65864B66798BCDC788D30A3B51F312
:105EE0000C04E0C15EBA0EBCC71EE5CD268A4EA6E4
:105EF00044EC974F1932DBCCE30228AD4DB66EDA95
:105F000048BE743F925FB1A335148F224CCA28302B
:105F10003A9FC1EF999A2302EA734FD243EE3CFEB7
:105F2000C3826190B08AC508D9B185680AA6EB3DE5
:105F3000288A2F44AFC2220D5CAF47AD22DA1E463D
:105F4000CEB6A8FF1D9CFB8E843639FDCE6B7F52EA
:105F5000818FBAC9CB134CB72045E34499F5537BE5
:105F60004B0CFD86E02086B35E38CC1DE21CA7A159
:105F7000E7AFE5E3919F87C1C8C1BEBFBF5394425D
:105F80007332C09476A20BC9F5AE24B2F119D79141
:105F9000D8463D489C14686893ECBF4349176C1F72
:105FA0004ADC1D995AEE1009095BA113A62160FF76
:105FB000AF6DED261F5D4F46EA40DC7E1E04F34BBD
:105FC00085A603F741AEEBB307A35D7BED54A4199F
:105FD000663FF47EDF08B66EB973E1161886453564
:105FE000919141AD6D6475C4B811C3491468FD0C3D
:105FF000E92A0D39679CB8F6501A59A694AA7D75FE
:00000001FF
